:0600000083018B018A015F
:06000600850186018C015A
:06000C009D018F0190012F
:060012009101920193012F
:060018009401950198011E
:06001E0099019A0183160E
:0600240010308500FF30E2
:06002A008600811764004E
:06003000A73081008312DD
:06003600850186010511A1
:06003C00051085101530CF
:060042009E009F019F0BD0
:0600480023289E0B232873
:06004E000F308605303082
:06005400860483160F3044
:06005A000605860083127A
:0600600005150511073033
:060066009E009F019F0BAC
:06006C0035289E0B35282B
:0600720005150511013027
:060078009E009F019F0B9A
:06007E003E289E0B3E2807
:060084000F30860520305C
:06008A00860405150511B6
:060090002830F1200830C9
:06009600F1200130F12011
:06009C000C30F1200630DB
:0600A200F1200730A5006B
:0600A8000C21A800083045
:0600AE00A5000C21A900D1
:0600B4000F30A5000C2135
:0600BA009B0003198628DB
:0600C0004530DE20453052
:0600C600DE202D30DE20DB
:0600CC004930DE204E3039
:0600D200DE204930DE20B3
:0600D8005430DE203A3036
:0600DE00DE2004210030C9
:0600E400A50025088900BB
:0600EA00AF208800152183
:0600F00040308038F120D1
:0600F600C02025089E2039
:0600FC00DE2004212508AE
:060102000F3C031C8628DF
:06010800A50A7328013076
:06010E00F120061C162A78
:06011400212982070034DE
:06011A0000340A34003439
:06012000003464340034D9
:060126000334E83400344C
:06012C00273410340134F9
:060132008634A0340F34F6
:060138004234403482074E
:06013E003034313432348C
:060144003334343435347D
:06014A003634373438346E
:0601500039344134423451
:060156004334443445343B
:06015C00463482070D3459
:06016200BC3436340D34FC
:06016800BB340A34003430
:06016E00153401340034D9
:060174000034FF34FF34EB
:06017A00FF34FF340034E5
:060180008316F0300604B6
:0601860086001830850020
:06018C008312051085142A
:0601920005150608F03916
:060198009B0005110000B0
:06019E000000051505112B
:0601A400060E0F391B04DA
:0601AA009B1BC02885101C
:0601B00083160F30060566
:0601B60086008312080020
:0601BC009600C0200F3088
:0601C20086051608F03965
:0601C800860485100514F9
:0601CE00051505110F30BC
:0601D4008605160EF0394D
:0601DA0086040515051165
:0601E00008009600C0209B
:0601E6000F30860516082B
:0601EC00F03986048510C5
:0601F200051005150511C2
:0601F8000F308605160E13
:0601FE00F039860405152E
:0602040005110800FF30A7
:06020A009E009F019F0B06
:0602100007299E0B0729DF
:0602160008008312250818
:06021C008900831608149E
:0602220083120808A6008B
:06022800080083168B1391
:06022E000815553089009F
:06023400AA3089008814C5
:06023A0088181D298B1736
:06024000080000308038C8
:06024600F120C02045304C
:06024C00DE204530DE203B
:060252005030DE205230A6
:06025800DE204F30DE2025
:06025E004D30DE202030CF
:06026400DE20403080386E
:06026A00F120C0204D3020
:06027000DE204F30DE200D
:060276004430DE2045309B
:06027C00DE202030DE2030
:060282003130DE202E30B9
:06028800DE203230DE2012
:06028E00042104210421FB
:06029400042104210421F5
:06029A00042106080F39E3
:0602A000031D21290130BD
:0602A600F120C020A501BB
:0602AC00A601A701061CDB
:0602B2006129A50A2508E0
:0602B8000F3C031CA50130
:0602BE0004212710861C3C
:0602C4006529A60A0421D1
:0602CA00061D6929A603D0
:0602D0000421861D8B29AC
:0602D60004212508890047
:0602DC0026088800152130
:0602E2000130F120C020F4
:0602E8002A30DE20533035
:0602EE00DE204130DE209D
:0602F4005630DE2045300B
:0602FA00DE204430DE208E
:060300002A30DE2004217A
:0603060004210421042182
:06030C0004210130F12084
:06031200C020A7014130EC
:06031800DE204430DE206F
:06031E004430DE205230E5
:06032400DE203A30DE206D
:06032A00271899290C219F
:0603300027142508F03936
:060336008E000E0E9E2059
:06033C00DE2025080F3948
:060342009E20DE20403089
:060348008038F120C02006
:06034E004430DE204130C6
:06035400DE205430DE2023
:06035A004130DE203A30C4
:06036000DE202608F03942
:060366008E000E0E9E2029
:06036C00DE2026080F3917
:060372009E20DE20003099
:060378008038F120C020D6
:06037E0058299B010C0848
:060384009C008B20031415
:06038A0098020318D329BC
:0603900003140130990284
:060396000318D329031433
:06039C0001309A02031873
:0603A200D3291B149C038B
:0603A8001C088B20031469
:0603AE0099020318E0298A
:0603B400031401309A025F
:0603BA000318E0291B14EA
:0603C0009C031C088B20C9
:0603C60003149A02031863
:0603CC00E9290314EA29EF
:0603D2001B0C00349B012E
:0603D8000C089C008B20C4
:0603DE0003109807031C48
:0603E400FE2903100130A8
:0603EA009907031CFE2927
:0603F000031001309A0722
:0603F600031CFE291B148C
:0603FC009C031C088B208D
:0604020003109907031C22
:060408000B2A0310013075
:06040E009A07031C0B2AF3
:060414001B149C031C08F0
:06041A008B2003149A0779
:06042000031C142A031462
:06042600152A1B0C003436
:06042C0011308C000930C4
:060432008D008E01063072
:060438009D00C021031825
:06043E00272A8E0A8D033F
:06044400031D1D2A033018
:06044A008C022A2AEB21BE
:0604500003308C020930AC
:060456008D0010301D07AF
:06045C009B009B031B083E
:0604620084000E088E016B
:0604680080009D0301303D
:06046E000C07031D1D2A0E
:0604740018088F0006309D
:06047A009D0025080605A7
:06048000A600A6194F2A98
:0604860007308038F12070
:06048C00C0202030DE203C
:060492000B308038F12060
:06049800C0202030DE2030
:06049E0000308038F1205F
:0604A400C0208608A5003F
:0604AA000F301D07840065
:0604B000000803195E2A9A
:0604B6003038DE20682A48
:0604BC00063003151D02CD
:0604C200031D662A203034
:0604C800DE20682A30303E
:0604CE00DE2086196D2AF4
:0604D4000230AA00742AA8
:0604DA000130AA000A3007
:0604E000A5000C21031D24
:0604E6007B2A2A08031521
:0604EC001D02031D7B2A26
:0604F2002E30DE20861909
:0604F8007F2A0530802A76
:0604FE00043003151D028D
:06050400031D862A2E30C3
:06050A00DE200930A5000F
:060510000C21031D942ADA
:06051600013003151D0277
:06051C00031D942A40308B
:060522008038F120C0202A
:060528009D0B552A0A306C
:06052E00A5000C21031DD5
:06053400A12A0F301D0793
:06053A00840000083038C7
:06054000DE202030DE2069
:060546004D30DE204830BC
:06054C00DE207A30DE2003
:0605520000308038F120AA
:0605580097018101000083
:06055E0000009D01C73002
:060564009E000B309F0019
:06056A000530A0008B012A
:0605700010308500831627
:060576001F308500831216
:06057C000B1DC32A970AC3
:060582000B11C62A000067
:06058800000000009E0BC4
:06058E00BE2AC7309E00EA
:060594009F0BBE2A0B3094
:06059A009F00A00BBE2A29
:0605A00082308E000B1DED
:0605A600D72A970A0B1191
:0605AC00DA2A0000000045
:0605B20000008E0BD22AAE
:0605B80028088E008E0BE6
:0605BE00DE2A29088E0070
:0605C40000008E0BE22A8C
:0605CA0003018600103061
:0605D000850083161730C0
:0605D600850083120B19E1
:0605DC00970A0B11010853
:0605E200990017089A00C1
:0605E8009B019B0A851532
:0605EE0085110B1101084C
:0605F400031119020319B6
:0605FA00F52A9B0A9B0993
:060600009B0A1B0A980092
:0606060010308500831690
:06060C000430850083129A
:060612000630A5000C21DA
:060618000319AE2B0619C8
:06061E00AE2B0519872B2D
:06062400003086180330CF
:06062A00A5000C210314E1
:0606300003111A02031C75
:06063600342B031D4D2BC7
:06063C00013086180430B5
:06064200A5000C210311CC
:0606480003141902031C5B
:06064E00342B031D4D2BAF
:060654000230861805309B
:06065A00A5000C210314B1
:060660001802031C342BFC
:060666004D2B0030861848
:06066C000330A5000C2183
:060672008F001A0893003E
:0606780001308618043079
:06067E00A5000C21900014
:0606840019089400023089
:06068A0086180530A500F2
:060690000C219100180886
:060696009500652B003009
:06069C0086180330A500E2
:0606A2000C2193001A0870
:0606A8008F0001308618EE
:0606AE000430A5000C2140
:0606B400940019089000FB
:0606BA0002308618053035
:0606C000A5000C219500CD
:0606C60018089100150860
:0606CC0003149102031863
:0606D200742B031401303B
:0606D80090020318742BD0
:0606DE00031401308F023D
:0606E4000318742B14083A
:0606EA0003149002031846
:0606F0007E2B0314013013
:0606F6008F0203187E2BA9
:0606FC0013088F020F0835
:060702009A0010089900A6
:0607080011089800162AFA
:06070E00023086180530E0
:06071400A5000C210310FA
:06071A009807031C9A2B56
:06072000031001309907EF
:06072600031C9A2B0310D6
:06072C0001309A07031CD6
:060732009A2B013086182D
:060738000430A5000C21B5
:06073E0003109907031CE3
:06074400A82B0310013098
:06074A009A07031CA82B16
:06075000030186180330CE
:06075600A5000C219A072A
:06075C00162AFF3FFF3FDB
:06076200FF3FFF3FFF3FD7
:06076800FF3FFF3FFF3FD1
:06076E00FF3FFF3FFF3FCB
:06077400FF3FFF3FFF3FC5
:06077A00FF3FFF3FFF3FBF
:06078000FF3FFF3FFF3FB9
:06078600FF3FFF3FFF3FB3
:06078C00FF3FFF3FFF3FAD
:06079200FF3FFF3FFF3FA7
:06079800FF3FFF3FFF3FA1
:06079E00FF3FFF3FFF3F9B
:0607A400FF3FFF3FFF3F95
:0607AA00FF3FFF3FFF3F8F
:0607B000FF3FFF3FFF3F89
:0607B600FF3FFF3FFF3F83
:0607BC00FF3FFF3FFF3F7D
:0607C200FF3FFF3FFF3F77
:0607C800FF3FFF3FFF3F71
:0607CE00FF3FFF3FFF3F6B
:0607D400FF3FFF3FFF3F65
:0607DA00FF3FFF3FFF3F5F
:0607E000FF3FFF3FFF3F59
:0607E600FF3FFF3FFF3F53
:0607EC00FF3FFF3FFF3F4D
:0607F200FF3FFF3FFF3F47
:0607F800FF3FFF3FFF3F41
:0207FE00FF3FBB
:084000000F000F000F000F007C
:02400E00F93F78
:00000001FF
